:020000040000FA
:06000000CA3001303A286D
:08000800A000030EA100831209
:100010008B1C32288B1031181428B11C3228643004
:10002000010203183128182800001628172818285C
:1000300019281A281B281C281D281E281F283110A3
:10004000B114A810031005190314AA0DA90DA80DC9
:10005000B00B322831152A08AF002908AE00280855
:10006000AD00B11081010B11210E8300A00E200EF6
:02007000090085
:0C007400203084008001840A80300402E7
:10008000031C3C281230B000DD2183160C3085059E
:1000900087018312850187010730990000309A009B
:1000A000103083168E008312603083168F00831207
:1000B0000030831691009F008312C83083168100A0
:1000C000831231309000003083168C008312103080
:1000D0008B00BC1B6D28851DEA22D12281018E0177
:1000E0008F010B118B100B108C018B178520311990
:1000F0009B20B30B8328031085190314B90DF0302E
:100100003902031941213023762864003118080090
:100110000B1D08000B11B11031141230B000051D79
:1001200096283214831601138312080032108316A6
:1001300001178312080031110130B7008B132030F2
:10014000370783169B001C141A088312A400A5000D
:10015000C030A5061030370783169B001C141A0800
:100160008312A3000030370783169B001C141A0863
:100170008312A2008B17321CC32822090339A20064
:10018000A309A409A50922082D02031D3B29230860
:100190002E02031D3B2924082F02031D3B29013099
:1001A0003702031DD8283D18D8283D143E14FF21DE
:1001B00002303702031DE128BD18E128BD143E14AA
:1001C0000E2203303702031DEA283D19EA283D15A7
:1001D0003E141A2204303702031DF328BD19F328F8
:1001E000BD153E14262205303702031DFC283D1A9A
:1001F000FC283D163E14352206303702031D052922
:10020000BD1A0529BD163E14442207303702031DCE
:100210000E293D1B0E293D173E145322083037028C
:10022000031D1729BD1B1729BD173E145E22093077
:100230003702031D20295E1820295E143E1469220E
:100240000A303702031D2929DE182929DE143E143D
:1002500074220B303702031D32295E1932295E15D4
:100260003E147F220C303702031D3B29DE193B2947
:10027000DE153E148A22B70A0D3037020318080033
:100280009E280130B600B300B400B500B700850168
:100290008701B1138520B30B892903108519031435
:1002A000B90DF03039020319B029B40B8929013096
:1002B0003702031995220230370203199A220330BC
:1002C000370203199F22043037020319A422053094
:1002D00037020319A922063037020319AE2207306C
:1002E00037020319B322083037020319B822093044
:1002F00037020319BD220A3037020319C2220B301C
:1003000037020319C7220C3037020319CC2296306A
:10031000B400311D4A293111321C93292D090339AA
:10032000AD00AE09AF092F1CB1132F1C4A29B11B18
:100330004A292E184A29B1178B1320303707BB00E2
:100340002F08BA00C82110303707BB002E08BA00AA
:10035000C82100303707BB002D08BA00C8218B1711
:1003600085018701B70AB6010D303702031C4A29FF
:10037000D12208003E1C08003E101030BB003D0892
:10038000BA00C8213030BB005E08BA00C82108009E
:100390008B133A0883161C159A0083123B088316A8
:1003A0009B0055309D00AA309D009C1464009C1851
:1003B000D6291C1183128B170800831600309B006E
:1003C0001C141A088312BC00831610309B001C14E6
:1003D0001A088312BD00831630309B001C141A08C3
:1003E0008312DE00FF30C800CA15CB15CC15CD1521
:1003F000CE15CF15D015D115D215D3150800C130A3
:10040000BD05FF30DE051130C405C0000030C2005C
:10041000C600BC185F14BC18DF140800C230BD054C
:10042000FF30DE050230C405C0000030C200C60047
:100430005F100800C430BD05FF30DE050630C4057E
:10044000C0000030C200C6005F100800C830BD0503
:10045000FF30DE051830C405C0000030C200C60001
:10046000BC185F14BC18DF140800D030BD05FF3085
:10047000DE053030C405C0000030C200C600BC1824
:100480005F14BC18DF140800E030BD05FF30DE0546
:100490003030C405C0002030C200C600BC185F1454
:1004A000BC18DF1408007F30BD05C030DE05C03049
:1004B000C505C1000030C300C7000800BF30BD053E
:1004C000C030DE053030C505C1000030C300C700B4
:1004D00008003F30BD05C130DE059030C505C100C4
:1004E0000030C300C70008003F30BD05C230DE0544
:1004F000C030C505C1000030C300C70008003F3050
:10050000BD05C430DE05C030C505C1000030C300E4
:10051000C70008003F30BD05C830DE05C030C50546
:10052000C1000030C300C70008001030850602304B
:100530008706080020308506003087060800213035
:1005400085060030870608000230850602308706DF
:100550000800003085060630870608000030850652
:100560000630870608000030870618308706080026
:1005700000308506213087060800003085060930E6
:10058000870608000030870618308706080000300C
:10059000870618308706080000308706183087065F
:1005A00008003D18FF21BD180E223D191A22BD1961
:1005B00026223D1A3522BD1A44223D1B5322BD1B63
:1005C0005E225E186922DE1874225E197F22DE190F
:1005D0008A220800B601B301B4013C1CF22ABC0116
:1005E000BC14F42ABC013C143C08B6006400F82A90
:1005F000F92AFA2AFB2AFC2AFF30B41B8500B41F13
:100600008501B30BF62AB40BF62A0310B60CB60814
:10061000031DF62A0030BB003C08BA00C8210800C0
:1006200005125C180516DC1C8512DC1885165C1D8D
:1006300005105C190514DC1D8510DC1985145C1E81
:1006400087105C1A8714DC1E0711DC1A07155C1F63
:1006500007105C1B0714DC1F8712DC1B87160800C1
:100660008F08031908008F0178308E00C80F622DA3
:10067000C80A441C602B461C512BCA1C422BCA01C1
:100680004A156E2B4A1D472BCA01CA156E2BCA1D6F
:100690004C2BCA014A166E2B4A1E6E2BCA01CA1475
:1006A0006E2B4A1D562BCA014A166E2BCA1D5B2B98
:1006B000CA014A166E2B4A1E6E2BCA01CA146E2B33
:1006C000CA1C652BCA014A156E2B4A1D6A2BCA012A
:1006D000CA156E2B4A1E6E2BCA014A15C41C952BD7
:1006E000C61C862BCB1C772BCB014B15A32B4B1D8C
:1006F0007C2BCB01CB15A32BCB1D812BCB014B1618
:10070000A32B4B1EA32BCB01CB14A32B4B1D8B2B4D
:10071000CB014B16A32BCB1D902BCB014B16A32B40
:100720004B1EA32BCB01CB14A32BCB1C9A2BCB01A1
:100730004B15A32B4B1D9F2BCB01CB15A32B4B1E76
:10074000A32BCB014B15441DCA2B461DBB2BCC1C28
:10075000AC2BCC014C15D82B4C1DB12BCC01CC159E
:10076000D82BCC1DB62BCC014C16D82B4C1ED82B1D
:10077000CC01CC14D82B4C1DC02BCC014C16D82B43
:10078000CC1DC52BCC014C16D82B4C1ED82BCC0124
:10079000CC14D82BCC1CCF2BCC014C15D82B4C1DFA
:1007A000D42BCC01CC15D82B4C1ED82BCC014C15FE
:1007B000C41D002CC61DF12BCD1CE22BCD014D1507
:1007C0005F130E2C4D1DE72BCD01CD150E2CCD1D2D
:1007D000EC2BCD014D160E2C4D1E0E2CCD01CD1443
:1007E0000E2C4D1DF62BCD014D160E2CCD1DFB2BC9
:1007F000CD014D160E2C4D1E0E2CCD01CD140E2C00
:10080000CD1C052CCD014D150E2C4D1D0A2CCD01F6
:10081000CD150E2C4D1E0E2CCD014D155F1B372C0A
:10082000441E372C461E282CCE1C192CCE014E15EA
:10083000452C4E1D1E2CCE01CE15452CCE1D232C35
:10084000CE014E16452C4E1E452CCE01CE14452C05
:100850004E1D2D2CCE014E16452CCE1D322CCE0118
:100860004E16452C4E1E452CCE01CE14452CCE1CCA
:100870003C2CCE014E15452C4E1D412CCE01CE15E3
:10088000452C4E1E452CCE014E15C41E6C2CC61E8A
:100890005D2CCF1C4E2CCF014F157A2C4F1D532CA5
:1008A000CF01CF157A2CCF1D582CCF014F167A2CA3
:1008B0004F1E7A2CCF01CF147A2C4F1D622CCF0102
:1008C0004F167A2CCF1D672CCF014F167A2C4F1E56
:1008D0007A2CCF01CF147A2CCF1C712CCF014F155D
:1008E0007A2C4F1D762CCF01CF157A2C4F1E7A2CE7
:1008F000CF014F15DF18A32C451EA32C471E942CA7
:10090000D01C852CD0015015B12C501D8A2CD00143
:10091000D015B12CD01D8F2CD0015016B12C501EEB
:10092000B12CD001D014B12C501D992CD0015016EF
:10093000B12CD01D9E2CD0015016B12C501EB12CC4
:10094000D001D014B12CD01CA82CD0015015B12C42
:10095000501DAD2CD001D015B12C501EB12CD001A2
:100960005015DF18DA2CC51EDA2CC71ECB2CD11C73
:10097000BC2CD1015115E82C511DC12CD101D11530
:10098000E82CD11DC62CD1015116E82C511EE82CA3
:10099000D101D114E82C511DD02CD1015116E82CD5
:1009A000D11DD52CD1015116E82C511EE82CD101B6
:1009B000D114E82CD11CDF2CD1015115E82C511D8C
:1009C000E42CD101D115E82C511EE82CD101511590
:1009D000DF18122D451F122D471F032DD21CF42C9A
:1009E000D2015215DF13202D521DF92CD201D21540
:1009F000202DD21DFE2CD2015216202D521E202D4C
:100A0000D201D214202D521D082DD2015216202DB4
:100A1000D21D0D2DD2015216202D521E202DD20195
:100A2000D214202DD21C172DD2015215202D521D6B
:100A30001C2DD201D215202D521E202DD20152156F
:100A4000DF184B2DDF1B4B2DC51F4B2DC71F3C2D1A
:100A5000D31C2D2DD3015315592D531D322DD301E8
:100A6000D315592DD31D372DD3015316592D531E90
:100A7000592DD301D314592D531D412DD301531694
:100A8000592DD31D462DD3015316592D531E592DC3
:100A9000D301D314592DD31C502DD3015315592DE7
:100AA000531D552DD301D315592D531E592DD30147
:100AB0005315BA214008C4004108C5005F18DF146F
:100AC0005F1CDF104808C9000C304A05031D0512E1
:100AD0000C304B05031D85120C304C05031D051011
:100AE0000C304D05031D85100C304E05031D87107D
:100AF0000C304F05031D07110C305005031D071066
:100B00000C305105031D87120C305205031D0712CE
:100B10000C305305031D871149080E020318BC2D24
:100B200012304A05031D051612304B05031D8516AC
:100B300012304C05031D051412304D05031D85149C
:100B400012304E05031D871412304F05031D071583
:100B500012305005031D071412305105031D87166E
:100B600012305205031D071612305305031D871559
:100B7000FF304802031908008F08031D0800852074
:100B800049080E02031CBC2D18304A05031D05122E
:100B900006304A05031D051618304B05031D851246
:100BA00006304B05031D851618304C05031D051036
:100BB00006304C05031D051418304D05031D851026
:100BC00006304D05031D851418304E05031D871092
:100BD00006304E05031D871418304F05031D0711FD
:100BE00006304F05031D071518305005031D07106B
:100BF00006305005031D071418305105031D8712D8
:100C000006305105031D871618305205031D0712C3
:100C100006305205031D071618305305031D8711B2
:0A0C200006305305031D8715080078
:084000000200030006000000AD
:02400E00CC33B1
:10420000010003000300030003000200020002009B
:104210000200000000000000000003000300030093
:10422000020000000000000000000000000000008C
:104230000000C000C000C000C000C000C000C0003E
:10424000FF00C300F300CF00FF00C300F300CF0066
:10425000FF00C300F300CF00FF00C300F300CF0056
:104260000100FF00FF00FF00FF00FF00FF00FF0054
:10427000FF00FF00FF00FF00FF00FF00FF00FF0046
:10428000FF000300FF00FF00FF00FF00FF00FF0032
:10429000FF00FF00FF00FF00FF00FF00FF00FF0026
:1042A000FF00C000FF00FF00FF00FF00FF00FF0055
:1042B000FF00FF00FF00FF00FF00FF00FF00FF0006
:1042C000FF00FF00FF00FF00FF00FF00FF00FF00F6
:1042D000FF00FF00FF00FF00FF00FF00FF00FF00E6
:1042E000FF00FF00FF00FF00FF00FF00FF00FF00D6
:1042F000FF00FF00FF00FF00FF00FF00FF00AA001B
:00000001FF
